:1064E9000A2A2A2A2A2A2A2A2A2A2A2A2A2A2A2A23
:1064F9002A2A20CFE0F0E0ECE5F2F0FB20E0E4E02E
:10650900EFF2E5F0E0202A2A2A2A2A2A2A2A2A2A28
:106519002A2A2A2A2A2A2A2A0A00312E204D4143C8
:1065290020E0E4F0E5F13A202025303262783A257E
:10653900303262783A25303262783A2530326278E0
:106549003A25303262783A25303262780A00322EA2
:1065590020495020E0E4F0E5F13A20202025627539
:106569002E2562752E2562752E2562750A00332E39
:1065790020D8EBFEE73A2020202020202025627534
:106589002E2562752E2562752E2562750A00342E18
:1065990020CCE0F1EAE020F1E5F2E83A2025627545
:1065A9002E2562752E2562752E2562750A00352EF7
:1065B90020495020E0E4F0E5F120F1E5F0E2E5F0D2
:1065C900E0313A202562752E2562752E2562752ED9
:1065D9002562750A00362E20495020E0E4F0E5F1E5
:1065E90020F1E5F0E2E5F0E0323A202562752E254A
:1065F90062752E2562752E2562750A00302E20CA15
:10660900EBFEF720E4EEF1F2F3EFE03A2025730A0E
:10661900000AC7C0CFC8D1DC20466C6173680A0084
:106629000AC7E0EFE8F1FC20E7E0E2E5F0F8E5ED84
:10663900E0210A00082008000A53696E636F6D495A
:1066490050205665722E20332E30205243202827A1
:106659002B2B2B272DE2F5EEE420E220EAEEEDF4D8
:10666900E8E3F3F0E0F2EEF029000A3E20CAEEED8D
:10667900F4E8E3F3F0E0F6E8EEEDEDFBE920F0E510
:10668900E6E8EC0A0A00203C493E20203A20CFEEF9
:10669900EAE0E7E0F2FC20EFE0F0E0ECE5F2F0FB05
:1066A9000A00203C536E3E203A20C7E0E4E0F2FCA9
:1066B90020EFE0F0E0ECE5F2F020276E270A002059
:1066C9003C4B3E20203A20C7E0E3F0F3E7E8F2FC38
:1066D90020EDEEE2F3FE20EAEEEDF42E20E8E720CD
:1066E900F4E0E9EBE00A00203C443E20203A20D0C7
:1066F900E0F1EFE5F7E0F2E0F2FC20EDEEE2F3FE87
:1067090020EAEEEDF42E0A00203C573E20203A20E4
:10671900C7E0EFE8F1E0F2FC20E8E7ECE5EDE5EDB4
:10672900E8FF0A00203C4C3E20203A20C7E0E3F075
:10673900F3E7E8F2FC20EFF0EEE3F0E0ECECF3280D
:10674900584D4F44454D290A00203C453E20203AEA
:1067590020C2FBF5EEE40A003E20C2E2E5E4E8F2DD
:10676900E520EAEEECE0EDE4F33A20000AC2E2E5C6
:10677900E4E8F2E520274D414320E0E4F0E5F15B50
:106789002562645D273A202530326278202D3E004B
:1067990078000AC2E2E5E4E8F2E52027495020E062
:1067A900E4E0EFF2E5F0E05B2562645D273A20253D
:1067B9006275202D3E0075000AC2E2E5E4E8F2E5C3
:1067C9002027D8EBFEE75B2562645D273A20256226
:1067D90075202D3E000AC2E2E5E4E8F2E52027CC67
:1067E900E0F1EAF3D1E5F2E85B2562645D273A203E
:1067F900256275202D3E000AC2E2E5E4E8F2E520B3
:1068090027495020F1E5F0E2E5F0E0315B256264CB
:106819005D273A20256275202D3E000AC2E2E5E493
:10682900E8F2E52027495020F1E5F0E2E5F0E03211
:106839005B2562645D273A20256275202D3E000A9A
:10684900C2E2E5E4E8F2E520EAEBFEF720E4EEF146
:10685900F2F3EFE028E4EE203720F1E8ECE2293A00
:106869000A2D3E000A204572726F72210A000AC879
:10687900C4C5D220C7C0CFC8D1DC2120C6C4C8D264
:10688900C521000AC7C0CFC8D1DC20C7C0C2C5D046
:10689900D8C5CDC0210A000A20000ACA20EFF0E8B5
:1068A900E5ECF320E3EEF2EEE2210A00C7E0EFF3B4
:1068B900F1F2E8F2E520EFE5F0E5E4E0F7F3204254
:1068C900494E20F4E0E9EBE020F120EFEEECEEF99F
:1068D900FCFE20584D4F44454D0A000A454F5421AE
:1068E9000A000AD4E0E9EB20E7E0E3F0F3E6E5ED9E
:1068F900210A00CEF8E8E1EAE0210A000AD4E0E939
:10690900EB20EFEEEBF3F7E5ED2120C7E0EFE8F13F
:10691900FC20E220454550524F4D210A003C4D4193
:10692900433D003C4130313D003C4130323D003C6B
:106939004130333D003C4130343D003C4130353D30
:10694900003C4130363D000ACAEEEDF4E8E3F3F0CD
:10695900E0F6E8FF20E7E0EFE8F1E0EDE0210A00EA
:10778400C2ADE4F5C9D2CDD2CCC2C9C2CAF5CDF5D9
:10779400CC75CBFF75CAB885CBCD85CACCD29ED269
:0A77A4009CD2CAC2ACC298C299225E
:077926003098FDAF99C298F3
:01792D002237
:0678E500127926EFF522E6
:0878EB008F993099FDC299222A
:1078D500AE07BE0A057F0D1278EBAF061278EB22D4
:1074AC007BFF7A6479E91269CB7BFF7A657923904B
:1074BC0061A2E0F535A3E0F536A3E0F537A3E0F5DE
:1074CC0038A3E0F539A3E0F53A1269CB7BFF7A6576
:1074DC0079579061A8E0F535A3E0F536A3E0F537D0
:1074EC00A3E0F5381269CB7BFF7A65797790619AC6
:1074FC00E0F535A3E0F536A3E0F537A3E0F5381257
:10750C0069CB7BFF7A65799790619EE0F535A3E0B6
:10751C00F536A3E0F537A3E0F5381269CB7BFF7A9B
:10752C006579B79061B1E0F535A3E0F536A3E0F5E8
:10753C0037A3E0F5381269CB7BFF7A6579DE906171
:10754C00B5E0F535A3E0F536A3E0F537A3E0F53863
:10755C001269CB7535017536617537CB7BFF7A6651
:05756C0079050269CB66
:067571008E298F2A8D2BEC
:10757700E4F530F531F52EF52FE52B60097BFF7A21
:1075870066791A1269CBE4F52CF52DE529C4F85470
:10759700F0C868FEE52AC4540F48FFC3E52D9FE5F0
:1075A7002C9E5031AE30AF31AD07AC067B10AF2FFC
:1075B700AE2E12772474102531F531E43530F530CD
:1075C7007410252FF52FE4352EF52E052DE52D709A
:1075D700BA052C80B6E529C4F854F0C868FEE52A38
:1075E700C4540F48C4F8540FC868FFEEC454F04899
:1075F700FEC3E52A9FFFE5299EAC30AD31AB07AF4F
:107607002FAE2E127724E52B60097BFF7A66792946
:037617001269CB2A
:01761A00224D
:0473DF007E677FBF87
:0473E3008E298F2A36
:1073E700E4F52B7400252BF582E43460F583E4F093
:1073F700052BE52BB408ECE4F52B127926EFF52CD9
:10740700640A6005E52CB40D0F7400252BF582E4A2
:107417003460F583E4F08044E52CB40824E52BD3ED
:107427009400402F7BFF7A66793D1269CB152B7448
:1074370000252BF582E43460F5837420F0152B804A
:10744700127400252BF582E43460F583E52CF0FFF8
:107457001278EB052BE52BC39408409EE52B7002B1
:10746700FF22852A82852983E493B4781E906000E1
:10747700E0FF1276F0EFC454F0FEC006906001E022
:10748700FF1276F0D0E02FF50880177531007532BE
:1074970000753300E4F5347B017A607900127103DB
:0474A7008F087F01CA
:0174AB0022BE
:10600300C2AFE58720E456907FFEE0B4FF047F0132
:1060130080027F00907FFDE0B4AA047E0180027EAF
:1060230000EE5FFF907FFFE0B455047E0180027EA7
:1060330000EE5F6019E4907FFDF0A3F0A3F0907F82
:10604300F0E0FEA3E0FF4E6005E4FD1275717BFFF7
:106053007A0079008B268A278928126FCE5387EF1F
:10606300127784C2987BFF7A6679411269CB3098A4
:106073000F7BFF7A0079008B268A278928126FCE3F
:10608300E4F525F523E4F5242098030264B412799A
:10609300268F22E522B42B051278EB0525E525C3CF
:1060A300940350030264A3E4F523E5232401FFE4EE
:1060B30033FE1277FD749A2523F582E43461F58368
:1060C300EFF00523E523C3943F40DFE4F523E52305
:1060D300247FFFE433FE1277FD74142523F582E455
:1060E3003461F583EFF00523E523C3948040DFE4B7
:1060F300906193F0E52570030264B47BFF7A6679BF
:10610300731269CB7BFF7A66798F1269CB7BFF7A37
:106113006679AB1269CB7BFF7A6679C81269CB7B50
:10612300FF7A6679F01269CB7BFF7A67791112697E
:10613300CB7BFF7A67792D1269CB7BFF7A67795224
:106143001269CB7BFF7A6779611269CB1278E5E537
:1061530022126FA8645C4463ED4561854964564B24
:1061630064504C618B5363F357645C6463ED656106
:10617300856964566B64506C618B7363F3770000BD
:1061830060F71274AC0260F71278E5E522126FA88B
:1061930063383061AC3161FD32623C33627B34621F
:1061A300BA3562F936000063E59061A274FAF0A390
:1061B30074CEF0A374CCF0752203E522C394064099
:1061C300030260F77BFF7A67797585223574A22510
:1061D30022F582E43461F583E0F5361269CB7E67FC
:1061E3007F991273E3EF600E74A22522F582E434E3
:1061F30061F583E508F0052280C0E4F522E522C3BA
:10620300940440030260F77BFF7A67799B8522350C
:1062130074A82522F582E43461F583E0F53612692A
:10622300CB1273DFEF600E74A82522F582E434618C
:10623300F583E508F0052280C4E4F522E522C39442
:106243000440030260F77BFF7A6779C185223574C6
:106253009A2522F582E43461F583E0F5361269CBA1
:106263001273DFEF600E749A2522F582E43461F530
:1062730083E508F0052280C4E4F522E522C39404F3
:1062830040030260F77BFF7A6779DE852235749ECF
:106293002522F582E43461F583E0F5361269CB12E9
:1062A30073DFEF600E749E2522F582E43461F5837B
:1062B300E508F0052280C4E4F522E522C3940440F6
:1062C300030260F77BFF7A68790085223574B12574
:1062D30022F582E43461F583E0F5361269CB12735B
:1062E300DFEF600E74B12522F582E43461F583E5B6
:1062F30008F0052280C4E4F522E522C39404400398
:106303000260F77BFF7A68792485223574B52522EC
:10631300F582E43461F583E0F5361269CB1273DF5D
:10632300EF600E74B52522F582E43461F583E50848
:10633300F0052280C47BFF7A6879481269CBE4F5C3
:106343002374CB2523F582E43461F583E4F005233C
:10635300E523B408ECE4F523127926EFF522640A69
:106363006005E522B40D0F74CB2523F582E4346177
:10637300F583E4F08044E522B40824E523D39400B4
:10638300402F7BFF7A66793D1269CB152374CB25A9
:1063930023F582E43461F5837420F01523801274AD
:1063A300CB2523F582E43461F583E522F0FF1278EF
:1063B300EB0523E523C39408409E9061CBE0642062
:1063C30060030260F7F523E523C3940840030260EA
:1063D300F774CB2523F582E43461F583E4F00523D8
:1063E30080E57BFF7A68796D805DE4F5250260F7CF
:1063F3007BFF7A6879771269CBE4F523E5232401DF
:10640300FFE433FE749A2523F582E43461F583E0D7
:10641300FD12785D0523E523C3943F40DFE4F523B4
:10642300E523247FFFE433FE74142523F582E4344B
:1064330061F583E0FD12785D0523E523C394804075
:10644300DF7BFF7A68798C1269CB0260F71272A73F
:106453000260F7126CC50260F77BFF7A6879A012BD
:1064630069CB906194E4F0A374FFF0E4F523C3E5F2
:106473002394D07480948740030260F7E522F4707C
:10648300030260F7E52270030260F71278AD8F22F2
:106493001278EBE522642170030260F7052380CEB6
:1064A300E525700D7BFFFAF98B26F527F528126F8A
:1064B300CE7F147E0012783E0524E524C394195040
:1064C3000302608B7F2E1278EB0523E523C3940A26
:1064D30050030260887BFF7A0079008B268A278924
:0664E30028126FCE80FEBE
:10783E00E4FDFCC3ED9FEC9E5014E4FBFA0BBB0081
:0E784E00010AEBF44A70F60DBD00010C80E556
:01785C002209
:1077D700E4FF7E0374142EF582E43460F583E02F12
:1077E700FF0EBE83EF74142EF582E43460F583E058
:0577F700FEC3EF9EFF40
:0177FC00226A
:1072A700752F60753017E4F52DF52EC2017BFF7A37
:1072B7006879A31269CB7BFF7A6879B51269CB200D
:1072C70098247F151278EBE4F529F52AC3E52A946B
:1072D70020E529648094CE50E62098E3052AE52A24
:1072E70070EA052980E6D200752C01E599B40409F6
:1072F7007BFF7A6879E41269CB3001030273B9C363
:10730700E52E94C0E52D945D40030273B9E4F52B97
:1073170020983AE4F529F52AAE29AF2AEE3395E00D
:10732700FDFCE47B407A9CF9F8D3126F2C400D20CA
:10733700980A052AE52A70E0052980DC20980E3096
:1073470000047F0680027F151278EB80C3C298E5A0
:107357002B7009E599B40404D20180177414252B06
:10736700F582E43460F583E599F0052BE52BC394AA
:1073770084409D1277D7EF600A7F151278EBC20021
:10738700027300D200906015E0B52C1E052CAE2FBD
:10739700AF30AD07AC067B80AF2EAE2D12772474CD
:1073A70080252EF52EE4352DF52D7F061278EB027C
:1073B70073007F201278EBE4F529F52A2098100551
:1073C7002AE52A70020529B420F2E529B44EED7B9F
:0873D700FF7A6879EB0269CB33
:1076F000EFC39430400BEFD394395005EF24D0FF03
:1077000022EFC39461400BEFD394665005EF24A998
:10771000FF22EFC39441400BEFD394465005EF2472
:04772000C9FF222259
:1078AD00906194E475F001126F16906194E0FEA35F
:0678BD00E0FF1277FD223E
:107895001278AD1276F0EFC454F0FEC0061278AD42
:0878A5001276F0D0E02FFF2263
:10769B001278AD906000EFF01278AD906001EFF0D2
:1076AB001278AD906002EFF01278AD906003EFF0BE
:1076BB001278AD906004EFF01278AD906005EFF0AA
:1076CB001278AD906006EFF01278AD906007EFF096
:1076DB00E4A3F0F531F532F533F5347B017A6079BB
:0576EB000012710322F2
:04761B008E2E8F2FF1
:10761F00906194E4F0A374FFF01278ADEF6069F419
:10762F006066852F82852E83E493B507EC75300154
:10763F00E52F2530F582E4352EF583E49360259010
:10764F006195E02530FF906194E03400FE1277FDE4
:10765F00E52F2530F582E4352EF583E493B5070445
:10766F00053080CCE52F2530F582E4352EF583E407
:10767F009370A6E53024FFFFE434FF9061948FF000
:0B768F00126F167E007F0122E4FEFF58
:01769A0022CD
:106CC5007BFF7A6879A31269CB9061D9126F77003F
:106CD500000000E4F529F52A209841D3E52A94001F
:106CE500E529940040199061D9126F53EF2401FFF3
:106CF500E43EFEE43DFDE43CFC9061D9126F6B7F00
:106D0500E07E937D047C009061D9126F5FD3126F92
:106D15004240C57BFF7A6879FC026F129061D912F7
:106D25006F77000000001279268F2DE52D643C60F9
:106D350011052AE52A70020529C394C0E529945D49
:106D45004096900000E52DF0752900752A0112790D
:106D5500268F2D852A82852983E52DF064216011F2
:106D6500052AE52A70020529C394D0E52994074030
:106D7500DD7BFF7A6979051269CBE52A2401F52CBB
:106D8500E43529F52BE4F529F52AC3E52A952CE503
:106D950029952B501EE4252AFFE5293401FE852A75
:106DA50082852983E0FD12785D052AE52A70DB05D9
:106DB5002980D77E697F2612761BEF4E60301278C8
:106DC500959061A2EFF01278959061A3EFF012789B
:106DD500959061A4EFF01278959061A5EFF0127887
:106DE500959061A6EFF01278959061A7EFF07E6916
:106DF5007F2C12761BEF4E60201278959061A8EFDC
:106E0500F01278959061A9EFF01278959061AAEF4C
:106E1500F01278959061ABEFF07E697F3212761BA8
:106E2500EF4E60201278959061B1EFF01278959051
:106E350061B2EFF01278959061B3EFF0127895900A
:106E450061B4EFF07E697F3812761BEF4E60201239
:106E550078959061B5EFF01278959061B6EFF012E4
:106E650078959061B7EFF01278959061B8EFF07E64
:106E7500697F3E12761BEF4E602012789590619ED9
:106E8500EFF012789590619FEFF01278959061A0E0
:106E9500EFF01278959061A1EFF07E697F4412764C
:106EA5001BEF4E602012789590619AEFF01278955D
:106EB50090619BEFF012789590619CEFF0127895B8
:106EC50090619DEFF07E697F4A12761BEF4E600858
:106ED50012769B9061B9EFF0E4F529F52AE52A24AD
:106EE50001FFE43529FE749A252AF582E43461F51B
:106EF50083E0FD12785D052AE52A70020529C39411
:106F050043E529940040D67BFF7A6979501269CB15
:016F15002259
:027724008B32A6
:10772600A2AF9202C2AF85A23353A2FE8E838F828E
:1077360005A28C838D8274091278C3E53253A2FEAA
:1077460043A2201278C553A2DF8533A2A20292AFCC
:01775600FF33
:01775700220F
:10781E00E4FDFCC3ED9FEC9E5015E4FBFA0BBB00A0
:0F782E00010ABA01F8BB90F50DBD00010C80E412
:01783D002228
:0D78F3004390014390025390FE5390FD22FC
:0D7900005390FD5390FE43900243900122EE
:0B787B00127758127886AF031277587E
:0E7886005390FD439002E5905408FF5390FD8F
:0178940022D1
:0D790D005390FD4390014390025390FD22E2
:07792E00AE071FEE70FA2204
:02775800AD077B
:10775A00E4FC5390FDEDA804088002C333D8FC3042
:10776A00E70543900180035390FE7F0512792E436B
:09777A0090020CBC08DC5390FDE8
:0177830022E3
:1077AE00E4FF5390FD7E07439002E59030E00D74A8
:1077BE0001A806088002C333D8FC42075390FD1E71
:0877CE00C3EE6480948050DFDB
:0177D6002290
:10785D00AB058F821278F37FA0127758127886AF1E
:0E786D008212787B1279007F0A7E0002781E5C
:0477FD00AB07AA0626
:107801001278F37FA012787B1278F37FA112775858
:0C7811001278861277AE12790D12790001
:01781D002248
:1078C300F922C002C004C00612FFF0D006D004D0D3
:0278D30002228F
:0360000002791A08
:0C791A0078FFE4F6D8FD7581450260039B
:106F1600C5F0F8A3E028F0C5F0F8E5821582700206
:066F26001583E038F022A3
:106F2C00EB9FF5F0EA9E42F0E99D42F0EC6480C8DC
:066F3C0064809845F0227C
:106F4200EB9FF5F0EA9E42F0E99D42F0E89C45F0A5
:016F5200221C
:0C6F5300E0FCA3E0FDA3E0FEA3E0FF22B1
:0C6F5F00E0F8A3E0F9A3E0FAA3E0FB22B5
:0C6F6B00ECF0A3EDF0A3EEF0A3EFF02299
:106F7700A8828583F0D083D082126F8E126F8E1213
:106F87006F8E126F8EE473E493A3C583C5F0C58338
:106F9700C8C582C8F0A3C583C5F0C583C8C582C864
:016FA70022C7
:106FA800D083D082F8E4937012740193700DA3A378
:106FB80093F8740193F5828883E47374029368608C
:066FC800EFA3A3A380DF8C
:066FCE008A838982E4734E
:10696900E5412435F8E605412278323009027835C7
:10697900E475F001127089026FD42002EB7F2ED2E8
:10698900028018EF540F2490D43440D4FF30060B02
:10699900EF24BFB41A0050032461FFE542600215D9
:1069A900420545E5457002054430090D7832E47524
:1069B900F001127089EF02701A0278D57403D209B6
:1069C9008003E4C209F5418B328A338934E4F54204
:1069D900F544F545E54260077F201269A480F57505
:1069E90043FFC203C202C204C205C207C208C20AE7
:1069F900126972FF700D3009057F001269B5AF4544
:106A0900AE4422B4255FC2D5C206126972FF24D0F2
:106A1900B40A00501A75F00A784230D50508B6FF55
:106A29000106C6A426F620D5047002D20580D92411
:106A3900CFB41A00EF5004C2E5D206026BB5D203F7
:106A490080C6D20280C0D20480BCD2D580BAD20717
:106A590080B47F201269A42004077401B542004064
:106A6900F1126969FF1269A40269DDD20AD20880AC
:106A790095126969FB126969FA126969F94A4B70D9
:106A89000679867A6C7BFF20042EE542602A7E0017
:106A99008E82758300126FED60060EEE654370F00D
:106AA900C2D5EBC0E0EAC0E0E9C0E0EE126BFCD071
:106AB900E0F9D0E0FAD0E0FB126FD4FF60AAEBC096
:106AC900E0EAC0E0E9C0E01269A4D0E02401F9D00D
:106AD900E03400FAD0E0FBE5430460DCD543D9801B
:106AE900877BFF7A6B79F8D204809C7910800279D0
:106AF90008C208C20A8008D2D5790A8004790AC274
:106B0900D5E543047002F543E4FAFDFEFF12696915
:106B1900FC7B08200313126969FD7B1030020A12FD
:106B29006969FE126969FF7B20EC3382D592D550E1
:106B390013C3E43002069FFFE49EFEE42003039D95
:106B4900FDE49CFCE4CBF8C203EC700CCFCECDCCB9
:106B5900E824F8F870F38017C3EF33FFEE33FEED46
:106B690033FDEC33FCEB33FB994002FB0FD8E9EB27
:106B7900300305F8D0E0C448B203C0E00AEC4D4E3A
:106B89004F78207B0070C2EAB5430040BCC0E012D8
:106B99006BFED0F0D0E0200304C4C0E0C4B203C04F
:106BA900F012698DD0F0D5F0EB0269DD126FA86A99
:106BB9007A536AF4586A4B4C6A47426AF84F6B0039
:0F6BC900446B00496A60436B06556AEA466AEA04
:106BD800456AEA476CA6506A4F2D6A532E6A762B8F
:106BE8006A57236A74206C8F2A6A0F4800006A6EFD
:106BF8003F3F3F00790AA2D5200514300709B91094
:106C0800020404B9080104A2D52008025001042096
:106C180004689204B542005034C0E07F2030051962
:106C28007F30A20472087207500F126C55C204C25A
:106C380008C207C20A7F30800F300703E9C0E0129C
:106C480069A4300703D0E0F9D0E0B542CC3007178B
:106C58007F30B9100C1269A47F583006077F7880FE
:106C680003B908031269A43004057F2D0269A47FC3
:106C780020200AF87F2B2008F322920480CF286E68
:106C8800756C6C2900D2031269693003F8C2037865
:106C98004230D50108F6026A0F2D5043495812694F
:106CA800692403B405004001E4906CA1931269952E
:0D6CB800743A126995D205754204026AF41F
:107103008B2E8A2F8930E4F53AF539F538F537F5C2
:1071130035F536E532453345316012EBC0E0EAC060
:10712300E0E9C0E0AB31AA32A933127099AB2E0566
:1071330030E530AA2F7002052F14F9126FD4F53BF6
:10714300C394094007E53BD3940D40E1E53B64203C
:1071530060DBE53BB42D054336038016E53BB42BDA
:1071630005433601800C74FF2530F53074FF352F4D
:10717300F52FE53460046410703FAB2EAA2FA930BD
:10718300126FD464306009E534702E75340A802997
:10719300900001126FEDFF64786004EFB45813435D
:1071A300360175341074022530F530E4352FF52F90
:1071B3008007E5347003753408AB2E0530E530AA3B
:1071C3002F7002052F14F9126FD4F53BC39461405D
:1071D3000AE53BD3947A5003533BDF74D0253BF548
:1071E3003BC3940A400CE53B9411406D74F9253B75
:1071F300F53BE53BD395345060433601853A3F85F3
:10720300393E85383D85373CAF347E00E4FCFDAB29
:107213003AAA39A938A83712702CC8ECC8C9EDC9E5
:10722300CAEECACBEFCBE4FCFDFEEB253BF53AEE11
:107233003AF539ED39F538EC38F537AF3AAE39ADC3
:1072430038FCAB3FAA3EA93DA83CD3126F42500382
:107253000271BC4336040271BCE53620E003E480CE
:107263002DE53245334531601EAB2EE53024FFF961
:10727300E52F34FFFAEBC0E0EAC0E0E9C0E0AB3150
:10728300AA32A933127099E53630E20774FFFFFE84
:10729300FDFC22E536AF3AAE39AD38AC3730E10309
:0472A30002707B22D8
:106FD400BB010689828A83E0225002E722BBFE02BB
:096FE400E32289828A83E49322EE
:106FED00BB010CE58229F582E5833AF583E0225059
:106FFD0006E92582F8E622BBFE06E92582F8E222A3
:0D700D00E58229F582E5833AF583E49322BC
:10701A00BB010689828A83F0225002F722BBFE0155
:02702A00F3224F
:10702C00E88FF0A4CC8BF0A42CFCE98EF0A42CFC03
:10703C008AF0EDA42CFCEA8EF0A4CDA8F08BF0A481
:10704C002DCC3825F0FDE98FF0A42CCD35F0FCEBE0
:10705C008EF0A4FEA9F0EB8FF0A4CFC5F02ECD39A5
:0F706C00FEE43CFCEAA42DCE35F0FDE43CFC2212
:0E707B00C3E49FFFE49EFEE49DFDE49CFC2226
:10708900FAE6FB0808E6F925F0F618E6CA3AF62208
:10709900BB011A89828A83D0F0D0E0F8D0E0F9D018
:1070A900E0FAD0E0FBE8C0E0C0F00270F15016E968
:1070B900F8D083D082D0E0F9D0E0FAD0E0FBC082EA
:1070C900C0830270E8BBFE16E9F8D083D082D0E015
:0F70D900F9D0E0FAD0E0FBC082C0830270FA2247
:0970E800EBF608EAF608E9F622CD
:0970F100EBF0A3EAF0A3E9F022A0
:0970FA00EBF208EAF208E9F222C7
:00000001FF
